:1000000054C0EBC308C2F6C36BC06AC069C068C005
:1000100067C066C065C064C063C062C00DC404032D
:10002000090422037700770077002E007200650034
:10003000630075007200730069006F006E002E008F
:100040006A00700010035500530042002D0032007A
:10005000330032001201100102000008C016E10551
:10006000000101020001090243000201008032097F
:100070000400000102020100052400100104240212
:100080000205240600010524010301070583030876
:1000900000FF09040100020A000000070501020236
:1000A0000000070581020800000011241FBECFE5F3
:1000B000D1E0DEBFCDBF10E0A0E6B0E0E4E9FBE0B8
:1000C00002C005900D92AC36B107D9F711E0ACE64D
:1000D000B0E001C01D92A034B107E1F7D2D458C5F9
:1000E0008FCFAC9A8BB780628BBF8BE480937D00FF
:1000F0008093A8008AE580937C008093A7000895F0
:100100001F93CF93DF93DC01162FEA01888184FFD0
:1001100005C0898198E88927898302C08AE5888398
:10012000AE014E5F5F4F212FFA018D9181932150D7
:100130001216DCF3CA01612F57D11C5F1883DF91BF
:10014000CF911F91089547EA50E0DADF08954CE718
:1001500050E0D6DF08951F93CF93DF9360918D0019
:10016000635067FDB3C080918A00CCE0D0E0C81B2B
:10017000D109CF56DF4F80918900803118F4CE012C
:1001800064D49EC08D3209F08BC0683009F098C0ED
:1001900083EC809371008AE58093600010926D007B
:1001A0008881807621F0CE0122D4282F66C09A81E2
:1001B00010927A008981882321F410927B0022E03A
:1001C00055C0853019F490938E004FC08630B9F534
:1001D0008B81813041F484E590E090938C00809392
:1001E0008B0022E128C0823021F4CE01EBD3282FEE
:1001F00022C08330F9F48A81882341F48EE190E0B3
:1002000090938C0080938B0024E015C0813041F4E2
:1002100082E290E090938C0080938B0022E20BC0EE
:10022000823041F484E490E090938C0080938B00C2
:1002300020E101C020E080E480936D001EC0883082
:1002400021F421E080E990E013C0893019F4909303
:1002500090000BC08A3011F421E008C08B3029F4E3
:100260008BE480937D008093A80020E08AE790E0F3
:1002700090938C0080938B0009C02F3F39F48881C4
:1002800087FD2E8180E880936D0006C08F818823D2
:1002900019F48E81821708F0822F8093610010C0BC
:1002A00080916D0087FF0CC0CE012CD48F3F21F4CC
:1002B0008EE18093600004C0882311F010926100E9
:1002C00080918D00181614F410928D0080916000BA
:1002D00084FF58C0809161008F3F09F453C0182FEC
:1002E000893008F018E0811B8093610080917100D3
:1002F00098E8892780937100112391F180916D0016
:1003000087FF08C082E790E0612F90D3182F8930D3
:1003100098F526C020918B0030918C0086FF0DC08F
:10032000A2E7B0E080E090E0F901E80FF91FE49166
:10033000ED9301961817C1F708C0912FD901E2E794
:10034000F0E08D9181939150E1F71150812F90E071
:100350001F5F0196820F931F90938C0080938B00F8
:1003600082E790E0612F40D0612F6C5F6C3041F0EC
:100370008FEF8093610004C08FEF809361006EE186
:100380006093600094E186B3887131F49150D9F79D
:1003900010928E001092880010E0992309F411E069
:1003A00080916C00811739F0112319F4F894A8D1C9
:1003B000789410936C00DF91CF911F910895A82F2E
:1003C000B92F80E090E041E050EA609530E009C04C
:1003D0002D9182279795879510F084279527305E79
:1003E000C8F36F5FA8F30895EADF8D939D93089596
:1003F000A6E088279927AA9569F00197E1F3B399B8
:10040000FCCFB39BFECF81E09927A6B3019611F0F4
:10041000A871D9F70895CF93CFB7CF93C395B39B66
:10042000E9F7B39B0BC0B39B09C0B39B07C0B39B59
:1004300005C0B39B03C0B39B01C0D8C00F92DF932C
:10044000C0918A00DD27CF56DF4F012EB39B03C03A
:10045000DF910F90E6CF2F930F931F934F932FEFC2
:100460004F6F06B303FB20F95F933F9350E03BE0EF
:1004700065C016B30126502953FDC89556B3012710
:1004800003FB25F92F7306B3B1F05027102713FB98
:1004900026F906B22230F0F000C016B3012703FBA4
:1004A00027F90126502906B22430E8F54F77206855
:1004B00016B30000F6CF50274F7D206206B2102FF2
:1004C000000000C006B300265029102713FB26F9B0
:1004D00006B2E2CF4F7B06B3206400C0DACF01261C
:1004E0005029187106B269F14E7F2160012F16B3B1
:1004F00028C0002650294D7F06B22260102F29C047
:10050000012650294B7F06B22460012F2DC016B35F
:1005100001265029477F2860000006B22EC04F7E7A
:1005200006B3206130C0422706B349930026502904
:10053000102706B24FEF13FB20F9297F16B379F28B
:10054000187159F10126502906B2012703FB21F940
:10055000237F06B371F2002650293150D0F006B245
:10056000102713FB22F9277E16B351F201265029DA
:10057000012703FB06B223F92F7C49F2000006B3E2
:10058000102713FB24F90026502906B22F7939F2DF
:1005900070CF10E21ABF00271CC03B503195C31B1F
:1005A000D04010E21ABF0881033C21F10B3411F155
:1005B000209188001981110F1213EDCF4A81441F39
:1005C000093669F10D3211F0013E29F74F7009F03B
:1005D000042F00938F003F915F914F911F910F91D6
:1005E0002F91DF910F90CAB7C5FD18CFCF91CFBF24
:1005F000CF91189520918F00222369F310918D00DF
:100600001123D1F53430D2F130938D00209389003D
:1006100010918A003BE0311B30938A002FC000917B
:100620008D0001304CF50AE54F7049F430916000BF
:1006300034FD25C000936000C1E7D0E024C0433002
:1006400049F030917C0034FD1AC000937C00CDE766
:10065000D0E019C03091A70034FD11C00093A7006D
:10066000C8EAD0E010C0052710E000C021C005276F
:1006700010E0C89508BB14C03AE501C032ED032E66
:10068000C0E0D0E032E017B31861C39A08B317BBDB
:1006900058E120E84FEF20FF052708BB2795179565
:1006A0001C3F28F700004552B0F720FF052727958B
:1006B00008BB17951C3FB8F629913A9561F7077E5C
:1006C00010918E00110F08BBC250D04011F0109352
:1006D000880010E21ABF086017B3177E402F477ECC
:1006E00054E05A95F1F708BB17BB48BB74CF80E0C4
:1006F00090E038D28F3F11F481B78C5F81BF0895AD
:10070000CF92DF92EF92FF920F931F93CF93DF93DD
:10071000E1B66EDE6C0188E981BF6ADE84539940E0
:1007200014F400E801C000E080E4F82EC0E0D0E05E
:10073000102F1F0D11BF5CDE9C0189E024333807A8
:100740000CF0102FF6942196C730D10511F0012F2F
:10075000EFCF2453394037FF03C0309521953F4FE9
:10076000C6018453994097FF03C0909581959F4F90
:100770008217930714F4E1BE27C0125011BF1E5F09
:100780007901C12FD0E0229610C032DE8453994007
:1007900097FF03C0909581959F4F8E159F0514F488
:1007A00011B77C0181B78F5F81BF81B790E0C81717
:1007B000D9075CF711BF80E090E0D4D1811721F018
:1007C00080E090E0612FD6D1DF91CF911F910F9102
:1007D000FF90EF90DF90CF900895B299189501BBEC
:1007E00005B50FBD09E00DBD07E000BF00E20BBF7E
:1007F00001B3189501BB0FB702BB0DB50A950DBD2E
:1008000079F00BB50695B29900680BBD13BB0FB517
:100810001EB5011B0FBD13B302B30FBF01B3189573
:1008200000BF04BD0BB50DBB00E40ABF00E60BBF63
:1008300002B30FBF01B3189501BBF09907C00BE4D9
:100840000EB90EBB08B50FB901B3189500E40EB987
:1008500000E003BF01B31895881F9795881F9795EF
:10086000881F9795881F9795881F9795881F97953C
:10087000881F9795881F9795892F08959C0181E07F
:1008800080BD80E888B9B99ABA988BB78F7B8BBF47
:100890001ABC13BE10BE80EE8EB984E58DB98FEF01
:1008A0008FB9B9017695679580E090E06C5E7041F4
:1008B0008C4F9F4F40E050E033D121502EBD8EB57C
:1008C00089BD1DBC8EB590E001969595879595954F
:1008D0008795819585BD95B58EB5891718F08EB52C
:1008E0008F5F85BD82E08ABD81E084BD90E499BFC1
:1008F00085B78C7F826085BF9ABF8BB780648BBFC2
:1009000010923E011092BB0010923C0110923D01EA
:10091000089584B5882379F49091BB00983058F4F9
:100920008DB3E92FF0E0ED54FF4F80839F5F9093EC
:10093000BB0081E084BD80917C0084FF12C0609187
:10094000BB00662321F480913F01882351F083EBA3
:1009500090E0FDDB8091BB00887080933F01109296
:10096000BB0083B7882369F5E0913E0180913D018A
:100970008E1739F1F0E0E454FF4F80816DDF209154
:100980003E012F5F2F7720933E0112BE9BE49EB95C
:100990001EBA982F9295907F9F6098BD8695F89487
:1009A0008FB983E083BF789480918D0087FF09C061
:1009B00080913D018095820F8F77823010F01092E8
:1009C0008D000895FC018381813049F484E590E035
:1009D00090938C0080938B0080915400089586E65C
:1009E00090E090938C0080938B0083E40895FC0149
:1009F0002081822F80768032B9F49181892F8052B4
:100A0000823010F48FEF0895923239F480916E00A5
:100A1000882319F482E080936E0027FD05C081E0F1
:100A200080933F0180E0089580E00895FC0180916B
:100A30006F00808380917000818312821382148200
:100A4000158288E0868387E00895DC010BC0E92FDA
:100A5000F0E0E454FF4F8D9180839F5F9F779093E8
:100A60003D01615090913D01662389F780913E01DF
:100A70008150891B8F77823018F48FEF80938D001F
:100A800008952EE088E190E00FB6F894A89581BD16
:100A90000FBE21BD2CDE87EE88BB88E187BBA89501
:100AA00084EC99E02CE931E0F9013197F1F70197F5
:100AB000D9F717BA80EC92E19093700080936F00A1
:100AC000DDDE0FDB10926E0010923F017894A89546
:100AD00042DB1FDF90916E009923C9F38091A7003C
:100AE00084FFF5CF923021F482E690E068E003C005
:100AF0008AE690E062E027DB80916E00815080936F
:100B00006E00E5CFFC01808180936F00818180932E
:100B1000700080916F0090917000B0DE81E00895C8
:100B2000A1E21A2EAA1BBB1BFD010DC0AA1FBB1FF1
:100B3000EE1FFF1FA217B307E407F50720F0A21B63
:100B4000B30BE40BF50B661F771F881F991F1A94D0
:100B500069F760957095809590959B01AC01BD01FA
:100B6000CF010895E199FECF1FBA8EBBE09A992775
:100B70008DB30895262FE199FECF1CBA1FBA8EBB04
:100B80002DBB0FB6F894E29AE19A0FBE0196089534
:040B9000F894FFCF07
:0C0B94005AFFA120000000000200030036
:00000001FF
